:1000000065280339AB000310AB0DAB0D83161F0839
:100010008F3930389F0083121F08F3392B040138C1
:100020009F00323030209F149F1814281E08B10002
:1000300083161E088312B00061288001840AFF3EE7
:10004000031D1D286128A801A700FF30A707031C76
:10005000A807031C61280330A600DF3031202528C3
:10006000A601E83EA500A609FC30031C3A28A50716
:1000700003183728A5070000A60F372825184028A1
:10008000A51C4428000044280800AA01A90110303A
:10009000AB00260DA90DAA0D2708A9022808031CEC
:1000A000280FAA0203185B282708A90728080318A5
:1000B000280FAA070310A50DA60DAB0B492825088C
:1000C000612883138312031308008501CE30831641
:1000D0008500803083129F00063083169F00073012
:1000E000831299002030840040301D200130A80088
:1000F000F43024200130D900053059020318882833
:1001000001308506A8002C302420D90A031D7C2844
:1001100002300120A3003108A4000310580D323E24
:10012000840023088000840A240880000E305802CE
:1001300003189C28D80A0429D801D101D001D9017B
:100140000F3059020318B6280310590D323E8400AF
:100150000008A300840A0008A4002308D00724088C
:100160000318013ED107D90A031DA0285108A60093
:100170005008A500A8010F30A7004520D000260890
:10018000D10001300120D2003108D30001305302E8
:10019000C230031952020318CE28D5288512051241
:1001A000D501D401FA302320C12851085302031C81
:1001B000DF28031DFF28500852020318FF28D40A25
:1001C0000319D50A0D305502031CF228031DEC2833
:1001D000AD305402031CF22805160B30D500EA306E
:1001E000D400F328051205145408143A5504031DCD
:1001F000FE2885160516C830232005120429D501CE
:10020000D4018512051005120530232088280729FE
:02400E00A43FCD
:00000001FF
